BL51 BANKED LINKER/LOCATER V5.01                                                        03/27/2012  18:03:32  PAGE 1


BL51 BANKED LINKER/LOCATER V5.01, INVOKED BY:
C:\KEIL\C51\BIN\BL51.EXE uc51all.obj TO uc51all


INPUT MODULES INCLUDED:
  uc51all.obj (UC51ALL)


LINK MAP OF MODULE:  uc51all (UC51ALL)


            TYPE    BASE      LENGTH    RELOCATION   SEGMENT NAME
            -----------------------------------------------------

            * * * * * * *   D A T A   M E M O R Y   * * * * * * *
            REG     0000H     0008H     ABSOLUTE     "REG BANK 0"

            * * * * * * *   C O D E   M E M O R Y   * * * * * * *
            CODE    0000H     06EDH     ABSOLUTE     



SYMBOL TABLE OF MODULE:  uc51all (UC51ALL)

  VALUE           TYPE          NAME
  ----------------------------------

  -------         MODULE        UC51ALL
  B:00A0H.0       SYMBOL        A0_8255
  B:00A0H.1       SYMBOL        A1_8255
  N:0055H         SYMBOL        ABUF
  D:00E0H         SYMBOL        ACC
  C:061CH         SYMBOL        ADCBIT
  C:02B0H         SYMBOL        ADC_SCR1
  C:02B9H         SYMBOL        ADC_SCR2
  C:05F0H         SYMBOL        ADC_SUBP
  N:0020H         SYMBOL        ADRS_9346
  C:0243H         SYMBOL        ADVAN_SCR1
  C:0251H         SYMBOL        ADVAN_SCR2
  C:0051H         SYMBOL        ADVLOOP
  N:0054H         SYMBOL        ATMP
  D:00F0H         SYMBOL        B
  C:048FH         SYMBOL        BACK
  N:0057H         SYMBOL        BOUNCE0
  N:0056H         SYMBOL        BOUNCE1
  C:03F7H         SYMBOL        CHECK_KEY
  C:040EH         SYMBOL        CHKLP
  C:036AH         SYMBOL        CHK_LCDBZY
  C:0540H         SYMBOL        CLK_PUS
  C:039CH         SYMBOL        CL_PC
  N:0053H         SYMBOL        CNY70
  N:0058H         SYMBOL        COUNTER
  N:0076H         SYMBOL        COUNT_0832
  N:007EH         SYMBOL        COUNT_164
  N:0074H         SYMBOL        COUNT_9346
  N:005FH         SYMBOL        CTRL55
  N:0073H         SYMBOL        DATA_HB
  N:0072H         SYMBOL        DATA_LB
BL51 BANKED LINKER/LOCATER V5.01                                                      03/27/2012  18:03:32  PAGE 2


  C:0516H         SYMBOL        DATA_PRO
  C:0408H         SYMBOL        DBLCHK
  C:0471H         SYMBOL        DCMNT2
  C:0476H         SYMBOL        DCMNT3
  C:047BH         SYMBOL        DCMNT4
  C:0480H         SYMBOL        DCMOVER
  C:0291H         SYMBOL        DCM_B
  C:028FH         SYMBOL        DCM_F
  C:0293H         SYMBOL        DCM_L
  C:0295H         SYMBOL        DCM_R
  C:0286H         SYMBOL        DCM_SCR1
  C:028EH         SYMBOL        DCM_SCR2
  C:046CH         SYMBOL        DCM_SUBP
  C:04C2H         SYMBOL        DL1
  C:04C5H         SYMBOL        DL2
  C:02DFH         SYMBOL        ENDPS
  C:05A4H         SYMBOL        ERASEWAIT
  C:0592H         SYMBOL        ERASE_DATA
  C:0586H         SYMBOL        EW_DIS
  C:057AH         SYMBOL        EW_ENA
  C:0481H         SYMBOL        FORWARD
  C:0076H         SYMBOL        FUNCT1
  C:0080H         SYMBOL        FUNCT11
  C:0084H         SYMBOL        FUNCT12
  C:008DH         SYMBOL        FUNCT13
  C:0092H         SYMBOL        FUNCT2
  C:009CH         SYMBOL        FUNCT21
  C:00ABH         SYMBOL        FUNCT22
  C:00B2H         SYMBOL        FUNCT3
  C:00BCH         SYMBOL        FUNCT31
  C:00CDH         SYMBOL        FUNCT32
  C:00D6H         SYMBOL        FUNCT4
  C:00E0H         SYMBOL        FUNCT41
  C:0103H         SYMBOL        FUNCT42
  C:010CH         SYMBOL        FUNCT5
  C:0118H         SYMBOL        FUNCT51
  C:0145H         SYMBOL        FUNCT52
  C:014CH         SYMBOL        FUNCT53
  C:0181H         SYMBOL        FUNCT54
  C:018AH         SYMBOL        FUNCT6
  C:01CEH         SYMBOL        FUNCT61
  C:01E0H         SYMBOL        FUNCT7
  C:01ECH         SYMBOL        FUNCT71
  C:01FFH         SYMBOL        FUNCT72
  C:0434H         SYMBOL        GREEN
  C:03F0H         SYMBOL        HAVE_STATE
  C:0000H         SYMBOL        INITIAL
  C:03F6H         SYMBOL        IS_KEY
  C:0067H         SYMBOL        JDG1
  C:006CH         SYMBOL        JDG2
  C:0071H         SYMBOL        JDG3
  C:0039H         SYMBOL        JDGKEY1
  C:005EH         SYMBOL        JDGKEY2
  N:0059H         SYMBOL        KEYDBL
  N:005AH         SYMBOL        KEYNUM
  B:0022H.0       SYMBOL        KEY_F
  C:02BAH         SYMBOL        LCD_CLS
BL51 BANKED LINKER/LOCATER V5.01                                                      03/27/2012  18:03:32  PAGE 3


  C:02C0H         SYMBOL        LCD_HOME
  C:02C6H         SYMBOL        LCD_LOCATE
  C:02D4H         SYMBOL        LCD_PRINTSTRING
  C:02E0H         SYMBOL        LCD_RDPOST
  B:0022H.1       SYMBOL        LED_FLG
  B:00A0H.3       SYMBOL        LED_GRN
  B:00A0H.2       SYMBOL        LED_RED
  C:049DH         SYMBOL        LEFT
  C:0028H         SYMBOL        LOOP
  C:0458H         SYMBOL        LOOP_164
  C:0213H         SYMBOL        MAIN_SCR1
  C:021BH         SYMBOL        MAIN_SCR2
  C:02A6H         SYMBOL        MEM_CODE
  C:0532H         SYMBOL        MEM_RD
  C:029DH         SYMBOL        MEM_SCR1
  C:02A5H         SYMBOL        MEM_SCR2
  C:0524H         SYMBOL        MEM_WR
  C:0225H         SYMBOL        MENU_SCR1
  C:0232H         SYMBOL        MENU_SCR2
  B:00A0H.6       SYMBOL        ML1
  B:00A0H.7       SYMBOL        ML2
  B:00A0H.4       SYMBOL        MR1
  B:00A0H.5       SYMBOL        MR2
  N:006FH         SYMBOL        MTR_CNT0
  N:006EH         SYMBOL        MTR_CNT1
  N:006DH         SYMBOL        MTR_TIME
  C:0447H         SYMBOL        NEXT164
  C:0042H         SYMBOL        NEXTJ1
  C:0047H         SYMBOL        NEXTJ2
  C:004CH         SYMBOL        NEXTJ3
  C:00FCH         SYMBOL        NEXTJG
  C:03FFH         SYMBOL        NEXTK
  C:00E9H         SYMBOL        NEXTSN
  C:0262H         SYMBOL        NI_SCR1
  C:026FH         SYMBOL        NI_SCR2
  C:02EFH         SYMBOL        NOTSEC
  C:0424H         SYMBOL        NOT_KEY
  C:027AH         SYMBOL        NS_SCR1
  C:0285H         SYMBOL        NS_SCR2
  C:062BH         SYMBOL        NUMBER_INPUT
  C:0439H         SYMBOL        NUMBER_SET
  C:0462H         SYMBOL        NUMCODE
  C:0297H         SYMBOL        OPS_SCR1
  C:029CH         SYMBOL        OPS_SCR2
  C:04D2H         SYMBOL        OPS_SUBP
  C:0454H         SYMBOL        OUT_H
  D:0090H         SYMBOL        P1
  D:00A0H         SYMBOL        P2
  D:00B0H         SYMBOL        P3
  N:005EH         SYMBOL        PA55
  N:005DH         SYMBOL        PB55
  N:005CH         SYMBOL        PC55
  N:005BH         SYMBOL        PCBIT
  C:0569H         SYMBOL        RDBIT
  C:0572H         SYMBOL        RDH
  C:0574H         SYMBOL        RDLP9346
  C:0565H         SYMBOL        RD_BYTE
BL51 BANKED LINKER/LOCATER V5.01                                                      03/27/2012  18:03:32  PAGE 4


  C:033CH         SYMBOL        RD_LCDCOM
  C:0382H         SYMBOL        RD_PA
  C:038AH         SYMBOL        RD_PB
  C:0618H         SYMBOL        READ_ADC
  C:05D5H         SYMBOL        READ_DATA
  C:042FH         SYMBOL        RED
  C:04ABH         SYMBOL        RIGHT
  C:04C2H         SYMBOL        RUN_DL
  B:00B0H.0       SYMBOL        S0832_CLK
  B:00B0H.1       SYMBOL        S0832_CS
  B:00B0H.3       SYMBOL        S0832_DI
  B:00B0H.4       SYMBOL        S0832_DO
  C:045CH         SYMBOL        S164CLK
  B:0090H.7       SYMBOL        S74CLK
  B:0090H.6       SYMBOL        S74CLR
  B:0090H.0       SYMBOL        S74DTA
  B:0090H.1       SYMBOL        S9346_CLK
  B:0090H.0       SYMBOL        S9346_CS
  B:0090H.2       SYMBOL        S9346_DI
  B:0090H.3       SYMBOL        S9346_DO
  C:03A6H         SYMBOL        SCAN_KEY
  C:02CDH         SYMBOL        SETB7
  C:01B5H         SYMBOL        SHOW_DT
  C:00F0H         SYMBOL        SHO_0
  C:00F7H         SYMBOL        SHO_1
  C:0054H         SYMBOL        SHO_ADVAN
  C:0206H         SYMBOL        SHO_LCM1
  C:020BH         SYMBOL        SHO_LCM2
  C:001EH         SYMBOL        SHO_MAIN
  C:002FH         SYMBOL        SHO_MENU
  C:04B9H         SYMBOL        STOP
  C:0392H         SYMBOL        ST_PC
  N:0052H         SYMBOL        TDL70
  C:042AH         SYMBOL        TEAM_SET
  N:0077H         SYMBOL        TEMP_0832
  N:007FH         SYMBOL        TEMP_164
  N:0075H         SYMBOL        TEMP_9346
  C:0270H         SYMBOL        TS_SCR1
  C:0279H         SYMBOL        TS_SCR2
  C:0550H         SYMBOL        WRBIT
  C:055DH         SYMBOL        WRH
  C:05ABH         SYMBOL        WRITE_DATA
  C:0561H         SYMBOL        WRLP9346
  C:05CCH         SYMBOL        WRWAIT
  C:054DH         SYMBOL        WR_BYTE
  C:0372H         SYMBOL        WR_CTRL
  C:0316H         SYMBOL        WR_LCDCMD
  C:02F0H         SYMBOL        WR_LCDDAT
  C:05FDH         SYMBOL        WR_OPCODE
  C:037AH         SYMBOL        WR_PA
  C:0546H         SYMBOL        WR_SB
  C:051DH         SYMBOL        Y70_DL
  C:0000H         LINE#         76
  C:0003H         LINE#         77
  C:0005H         LINE#         80
  C:0008H         LINE#         81
  C:000AH         LINE#         83
BL51 BANKED LINKER/LOCATER V5.01                                                      03/27/2012  18:03:32  PAGE 5


  C:000DH         LINE#         84
  C:000FH         LINE#         86
  C:0012H         LINE#         87
  C:0014H         LINE#         89
  C:0016H         LINE#         90
  C:0018H         LINE#         92
  C:001AH         LINE#         93
  C:001CH         LINE#         95
  C:001EH         LINE#         98
  C:0021H         LINE#         99
  C:0023H         LINE#         100
  C:0026H         LINE#         101
  C:0028H         LINE#         104
  C:002AH         LINE#         105
  C:002CH         LINE#         106
  C:002FH         LINE#         109
  C:0032H         LINE#         110
  C:0034H         LINE#         111
  C:0037H         LINE#         112
  C:0039H         LINE#         114
  C:003BH         LINE#         115
  C:003DH         LINE#         116
  C:0040H         LINE#         117
  C:0042H         LINE#         118
  C:0045H         LINE#         119
  C:0047H         LINE#         120
  C:004AH         LINE#         121
  C:004CH         LINE#         122
  C:004FH         LINE#         123
  C:0051H         LINE#         126
  C:0054H         LINE#         129
  C:0057H         LINE#         130
  C:0059H         LINE#         131
  C:005CH         LINE#         132
  C:005EH         LINE#         134
  C:0060H         LINE#         135
  C:0062H         LINE#         136
  C:0065H         LINE#         137
  C:0067H         LINE#         138
  C:006AH         LINE#         139
  C:006CH         LINE#         140
  C:006FH         LINE#         141
  C:0071H         LINE#         142
  C:0074H         LINE#         143
  C:0076H         LINE#         146
  C:0079H         LINE#         147
  C:007BH         LINE#         148
  C:007EH         LINE#         149
  C:0080H         LINE#         151
  C:0082H         LINE#         152
  C:0084H         LINE#         154
  C:0086H         LINE#         155
  C:0088H         LINE#         156
  C:008BH         LINE#         157
  C:008DH         LINE#         159
  C:0090H         LINE#         160
  C:0092H         LINE#         163
BL51 BANKED LINKER/LOCATER V5.01                                                      03/27/2012  18:03:32  PAGE 6


  C:0095H         LINE#         164
  C:0097H         LINE#         165
  C:009AH         LINE#         166
  C:009CH         LINE#         168
  C:009EH         LINE#         169
  C:00A0H         LINE#         170
  C:00A1H         LINE#         171
  C:00A3H         LINE#         172
  C:00A5H         LINE#         173
  C:00A7H         LINE#         174
  C:00A9H         LINE#         175
  C:00ABH         LINE#         177
  C:00ADH         LINE#         178
  C:00B0H         LINE#         179
  C:00B2H         LINE#         182
  C:00B5H         LINE#         183
  C:00B7H         LINE#         184
  C:00BAH         LINE#         185
  C:00BCH         LINE#         187
  C:00BEH         LINE#         188
  C:00C0H         LINE#         189
  C:00C2H         LINE#         190
  C:00C3H         LINE#         191
  C:00C5H         LINE#         192
  C:00C7H         LINE#         193
  C:00C9H         LINE#         194
  C:00CBH         LINE#         195
  C:00CDH         LINE#         197
  C:00CFH         LINE#         198
  C:00D2H         LINE#         199
  C:00D4H         LINE#         200
  C:00D6H         LINE#         203
  C:00D9H         LINE#         204
  C:00DBH         LINE#         205
  C:00DEH         LINE#         206
  C:00E0H         LINE#         208
  C:00E2H         LINE#         209
  C:00E4H         LINE#         210
  C:00E5H         LINE#         211
  C:00E7H         LINE#         212
  C:00E9H         LINE#         213
  C:00EBH         LINE#         214
  C:00ECH         LINE#         215
  C:00EEH         LINE#         216
  C:00F0H         LINE#         217
  C:00F3H         LINE#         218
  C:00F5H         LINE#         219
  C:00F7H         LINE#         220
  C:00FAH         LINE#         221
  C:00FCH         LINE#         222
  C:00FEH         LINE#         224
  C:0101H         LINE#         225
  C:0103H         LINE#         227
  C:0105H         LINE#         228
  C:0107H         LINE#         229
  C:010AH         LINE#         230
  C:010CH         LINE#         233
BL51 BANKED LINKER/LOCATER V5.01                                                      03/27/2012  18:03:32  PAGE 7


  C:010FH         LINE#         234
  C:0111H         LINE#         235
  C:0114H         LINE#         236
  C:0116H         LINE#         237
  C:0118H         LINE#         239
  C:011AH         LINE#         240
  C:011CH         LINE#         241
  C:011DH         LINE#         242
  C:011FH         LINE#         243
  C:0121H         LINE#         244
  C:0123H         LINE#         245
  C:0126H         LINE#         246
  C:0128H         LINE#         247
  C:0129H         LINE#         248
  C:012BH         LINE#         249
  C:012DH         LINE#         250
  C:012FH         LINE#         252
  C:0131H         LINE#         253
  C:0133H         LINE#         254
  C:0135H         LINE#         255
  C:0136H         LINE#         256
  C:0138H         LINE#         257
  C:013AH         LINE#         258
  C:013CH         LINE#         259
  C:013EH         LINE#         260
  C:013FH         LINE#         261
  C:0141H         LINE#         262
  C:0143H         LINE#         263
  C:0145H         LINE#         264
  C:0147H         LINE#         265
  C:014AH         LINE#         266
  C:014CH         LINE#         267
  C:014EH         LINE#         268
  C:0151H         LINE#         270
  C:0153H         LINE#         271
  C:0155H         LINE#         272
  C:0156H         LINE#         273
  C:0158H         LINE#         274
  C:015BH         LINE#         275
  C:015CH         LINE#         276
  C:015EH         LINE#         277
  C:0160H         LINE#         278
  C:0163H         LINE#         279
  C:0165H         LINE#         280
  C:0166H         LINE#         281
  C:0168H         LINE#         282
  C:016AH         LINE#         284
  C:016CH         LINE#         285
  C:016DH         LINE#         286
  C:016FH         LINE#         287
  C:0172H         LINE#         288
  C:0173H         LINE#         289
  C:0175H         LINE#         290
  C:0177H         LINE#         291
  C:017AH         LINE#         292
  C:017CH         LINE#         293
  C:017DH         LINE#         294
BL51 BANKED LINKER/LOCATER V5.01                                                      03/27/2012  18:03:32  PAGE 8


  C:017FH         LINE#         295
  C:0181H         LINE#         297
  C:0183H         LINE#         298
  C:0185H         LINE#         299
  C:0188H         LINE#         300
  C:018AH         LINE#         303
  C:018DH         LINE#         304
  C:018FH         LINE#         305
  C:0192H         LINE#         306
  C:0194H         LINE#         308
  C:0196H         LINE#         309
  C:0198H         LINE#         310
  C:019BH         LINE#         311
  C:019CH         LINE#         312
  C:019DH         LINE#         314
  C:019FH         LINE#         315
  C:01A2H         LINE#         316
  C:01A3H         LINE#         317
  C:01A4H         LINE#         319
  C:01A6H         LINE#         320
  C:01A9H         LINE#         321
  C:01AAH         LINE#         322
  C:01ADH         LINE#         323
  C:01AEH         LINE#         324
  C:01AFH         LINE#         326
  C:01B0H         LINE#         327
  C:01B2H         LINE#         328
  C:01B4H         LINE#         329
  C:01B5H         LINE#         331
  C:01B8H         LINE#         332
  C:01B9H         LINE#         333
  C:01BAH         LINE#         334
  C:01BCH         LINE#         335
  C:01BEH         LINE#         336
  C:01C1H         LINE#         337
  C:01C3H         LINE#         338
  C:01C4H         LINE#         339
  C:01C5H         LINE#         340
  C:01C7H         LINE#         341
  C:01C9H         LINE#         342
  C:01CCH         LINE#         343
  C:01CEH         LINE#         345
  C:01D0H         LINE#         346
  C:01D2H         LINE#         347
  C:01D4H         LINE#         348
  C:01D5H         LINE#         349
  C:01D7H         LINE#         351
  C:01D9H         LINE#         352
  C:01DBH         LINE#         353
  C:01DEH         LINE#         354
  C:01E0H         LINE#         357
  C:01E3H         LINE#         358
  C:01E5H         LINE#         359
  C:01E8H         LINE#         360
  C:01EAH         LINE#         361
  C:01ECH         LINE#         363
  C:01EEH         LINE#         364
BL51 BANKED LINKER/LOCATER V5.01                                                      03/27/2012  18:03:32  PAGE 9


  C:01EFH         LINE#         365
  C:01F1H         LINE#         366
  C:01F3H         LINE#         367
  C:01F4H         LINE#         368
  C:01F6H         LINE#         369
  C:01F8H         LINE#         370
  C:01FAH         LINE#         371
  C:01FCH         LINE#         372
  C:01FDH         LINE#         373
  C:01FFH         LINE#         375
  C:0201H         LINE#         376
  C:0204H         LINE#         377
  C:0206H         LINE#         380
  C:0208H         LINE#         381
  C:020AH         LINE#         382
  C:020BH         LINE#         384
  C:020CH         LINE#         385
  C:020EH         LINE#         386
  C:0210H         LINE#         387
  C:0212H         LINE#         388
  C:02BAH         LINE#         426
  C:02BDH         LINE#         427
  C:02BFH         LINE#         428
  C:02C0H         LINE#         431
  C:02C3H         LINE#         432
  C:02C5H         LINE#         433
  C:02C6H         LINE#         436
  C:02C8H         LINE#         437
  C:02CBH         LINE#         438
  C:02CDH         LINE#         439
  C:02CFH         LINE#         440
  C:02D1H         LINE#         441
  C:02D3H         LINE#         442
  C:02D4H         LINE#         445
  C:02D5H         LINE#         446
  C:02D6H         LINE#         447
  C:02D8H         LINE#         448
  C:02DAH         LINE#         449
  C:02DCH         LINE#         450
  C:02DDH         LINE#         451
  C:02DFH         LINE#         452
  C:02E0H         LINE#         455
  C:02E2H         LINE#         456
  C:02E4H         LINE#         457
  C:02E6H         LINE#         458
  C:02E8H         LINE#         459
  C:02EBH         LINE#         460
  C:02EDH         LINE#         461
  C:02EFH         LINE#         462
  C:02F0H         LINE#         465
  C:02F2H         LINE#         466
  C:02F5H         LINE#         467
  C:02F7H         LINE#         468
  C:02FAH         LINE#         469
  C:02FCH         LINE#         470
  C:02FFH         LINE#         471
  C:0301H         LINE#         472
BL51 BANKED LINKER/LOCATER V5.01                                                      03/27/2012  18:03:32  PAGE 10


  C:0304H         LINE#         473
  C:0306H         LINE#         474
  C:0309H         LINE#         475
  C:030BH         LINE#         476
  C:030EH         LINE#         477
  C:0310H         LINE#         478
  C:0313H         LINE#         479
  C:0315H         LINE#         480
  C:0316H         LINE#         483
  C:0318H         LINE#         484
  C:031BH         LINE#         485
  C:031DH         LINE#         486
  C:0320H         LINE#         487
  C:0322H         LINE#         488
  C:0325H         LINE#         489
  C:0327H         LINE#         490
  C:032AH         LINE#         491
  C:032CH         LINE#         492
  C:032FH         LINE#         493
  C:0331H         LINE#         494
  C:0334H         LINE#         495
  C:0336H         LINE#         496
  C:0339H         LINE#         497
  C:033BH         LINE#         498
  C:033CH         LINE#         501
  C:033FH         LINE#         502
  C:0341H         LINE#         504
  C:0344H         LINE#         505
  C:0346H         LINE#         506
  C:0349H         LINE#         507
  C:034BH         LINE#         508
  C:034EH         LINE#         509
  C:0350H         LINE#         510
  C:0352H         LINE#         511
  C:0355H         LINE#         512
  C:0358H         LINE#         513
  C:035AH         LINE#         514
  C:035DH         LINE#         515
  C:035FH         LINE#         516
  C:0362H         LINE#         517
  C:0364H         LINE#         519
  C:0367H         LINE#         520
  C:0369H         LINE#         521
  C:036AH         LINE#         524
  C:036CH         LINE#         525
  C:036EH         LINE#         526
  C:0371H         LINE#         527
  C:0372H         LINE#         531
  C:0374H         LINE#         532
  C:0376H         LINE#         533
  C:0378H         LINE#         534
  C:0379H         LINE#         535
  C:037AH         LINE#         538
  C:037CH         LINE#         539
  C:037EH         LINE#         540
  C:0380H         LINE#         541
  C:0381H         LINE#         542
BL51 BANKED LINKER/LOCATER V5.01                                                      03/27/2012  18:03:32  PAGE 11


  C:0382H         LINE#         545
  C:0384H         LINE#         546
  C:0386H         LINE#         547
  C:0387H         LINE#         548
  C:0389H         LINE#         549
  C:038AH         LINE#         552
  C:038CH         LINE#         553
  C:038EH         LINE#         554
  C:038FH         LINE#         555
  C:0391H         LINE#         556
  C:0392H         LINE#         559
  C:0394H         LINE#         560
  C:0396H         LINE#         561
  C:0398H         LINE#         562
  C:0399H         LINE#         563
  C:039AH         LINE#         564
  C:039BH         LINE#         565
  C:039CH         LINE#         568
  C:039EH         LINE#         569
  C:03A0H         LINE#         570
  C:03A2H         LINE#         571
  C:03A3H         LINE#         572
  C:03A4H         LINE#         573
  C:03A5H         LINE#         574
  C:03A6H         LINE#         577
  C:03A9H         LINE#         578
  C:03ABH         LINE#         581
  C:03AEH         LINE#         582
  C:03B0H         LINE#         583
  C:03B3H         LINE#         584
  C:03B5H         LINE#         585
  C:03B7H         LINE#         586
  C:03B9H         LINE#         587
  C:03BCH         LINE#         589
  C:03BFH         LINE#         590
  C:03C1H         LINE#         591
  C:03C4H         LINE#         592
  C:03C6H         LINE#         593
  C:03C8H         LINE#         594
  C:03CAH         LINE#         595
  C:03CDH         LINE#         597
  C:03D0H         LINE#         598
  C:03D2H         LINE#         599
  C:03D5H         LINE#         600
  C:03D7H         LINE#         601
  C:03D9H         LINE#         602
  C:03DBH         LINE#         603
  C:03DEH         LINE#         605
  C:03E1H         LINE#         606
  C:03E3H         LINE#         607
  C:03E6H         LINE#         608
  C:03E8H         LINE#         609
  C:03EAH         LINE#         610
  C:03ECH         LINE#         611
  C:03EFH         LINE#         613
  C:03F0H         LINE#         616
  C:03F2H         LINE#         617
BL51 BANKED LINKER/LOCATER V5.01                                                      03/27/2012  18:03:32  PAGE 12


  C:03F5H         LINE#         618
  C:03F6H         LINE#         621
  C:03F7H         LINE#         624
  C:03FAH         LINE#         625
  C:03FCH         LINE#         626
  C:03FFH         LINE#         627
  C:0400H         LINE#         628
  C:0402H         LINE#         629
  C:0404H         LINE#         630
  C:0407H         LINE#         631
  C:0408H         LINE#         633
  C:040BH         LINE#         634
  C:040EH         LINE#         635
  C:0411H         LINE#         636
  C:0414H         LINE#         637
  C:0417H         LINE#         638
  C:0419H         LINE#         639
  C:041CH         LINE#         640
  C:041EH         LINE#         641
  C:0421H         LINE#         642
  C:0423H         LINE#         643
  C:0424H         LINE#         644
  C:0426H         LINE#         645
  C:0429H         LINE#         646
  C:042AH         LINE#         649
  C:042DH         LINE#         650
  C:042FH         LINE#         653
  C:0431H         LINE#         654
  C:0433H         LINE#         655
  C:0434H         LINE#         658
  C:0436H         LINE#         659
  C:0438H         LINE#         660
  C:0439H         LINE#         663
  C:043CH         LINE#         664
  C:043DH         LINE#         665
  C:043FH         LINE#         666
  C:0442H         LINE#         667
  C:0444H         LINE#         668
  C:0445H         LINE#         669
  C:0447H         LINE#         672
  C:0449H         LINE#         673
  C:044AH         LINE#         674
  C:044CH         LINE#         676
  C:044EH         LINE#         677
  C:0450H         LINE#         678
  C:0452H         LINE#         679
  C:0454H         LINE#         680
  C:0456H         LINE#         681
  C:0458H         LINE#         684
  C:045BH         LINE#         685
  C:045CH         LINE#         688
  C:045EH         LINE#         689
  C:045FH         LINE#         690
  C:0461H         LINE#         691
  C:046CH         LINE#         698
  C:046FH         LINE#         699
  C:0471H         LINE#         700
BL51 BANKED LINKER/LOCATER V5.01                                                      03/27/2012  18:03:32  PAGE 13


  C:0474H         LINE#         701
  C:0476H         LINE#         702
  C:0479H         LINE#         703
  C:047BH         LINE#         704
  C:047EH         LINE#         705
  C:0480H         LINE#         707
  C:0481H         LINE#         710
  C:0484H         LINE#         711
  C:0486H         LINE#         712
  C:0488H         LINE#         713
  C:048AH         LINE#         714
  C:048CH         LINE#         715
  C:048EH         LINE#         716
  C:048FH         LINE#         719
  C:0492H         LINE#         720
  C:0494H         LINE#         721
  C:0496H         LINE#         722
  C:0498H         LINE#         723
  C:049AH         LINE#         724
  C:049CH         LINE#         725
  C:049DH         LINE#         728
  C:04A0H         LINE#         729
  C:04A2H         LINE#         730
  C:04A4H         LINE#         731
  C:04A6H         LINE#         732
  C:04A8H         LINE#         733
  C:04AAH         LINE#         734
  C:04ABH         LINE#         737
  C:04AEH         LINE#         738
  C:04B0H         LINE#         739
  C:04B2H         LINE#         740
  C:04B4H         LINE#         741
  C:04B6H         LINE#         742
  C:04B8H         LINE#         743
  C:04B9H         LINE#         746
  C:04BBH         LINE#         747
  C:04BDH         LINE#         748
  C:04BFH         LINE#         749
  C:04C1H         LINE#         750
  C:04C2H         LINE#         753
  C:04C5H         LINE#         754
  C:04C8H         LINE#         755
  C:04CBH         LINE#         756
  C:04CEH         LINE#         757
  C:04D1H         LINE#         758
  C:04D2H         LINE#         760
  C:04D5H         LINE#         762
  C:04D8H         LINE#         763
  C:04DAH         LINE#         764
  C:04DDH         LINE#         765
  C:04DFH         LINE#         766
  C:04E1H         LINE#         767
  C:04E3H         LINE#         768
  C:04E5H         LINE#         770
  C:04E8H         LINE#         771
  C:04EAH         LINE#         772
  C:04EDH         LINE#         773
BL51 BANKED LINKER/LOCATER V5.01                                                      03/27/2012  18:03:32  PAGE 14


  C:04EFH         LINE#         774
  C:04F1H         LINE#         775
  C:04F3H         LINE#         776
  C:04F5H         LINE#         778
  C:04F8H         LINE#         779
  C:04FAH         LINE#         780
  C:04FDH         LINE#         781
  C:04FFH         LINE#         782
  C:0501H         LINE#         783
  C:0503H         LINE#         784
  C:0505H         LINE#         786
  C:0508H         LINE#         787
  C:050AH         LINE#         788
  C:050DH         LINE#         789
  C:050FH         LINE#         790
  C:0511H         LINE#         791
  C:0513H         LINE#         792
  C:0515H         LINE#         794
  C:0516H         LINE#         797
  C:0519H         LINE#         798
  C:051CH         LINE#         799
  C:051DH         LINE#         802
  C:0520H         LINE#         803
  C:0523H         LINE#         804
  C:0524H         LINE#         808
  C:0526H         LINE#         809
  C:0528H         LINE#         810
  C:052AH         LINE#         811
  C:052CH         LINE#         813
  C:052FH         LINE#         814
  C:0531H         LINE#         815
  C:0532H         LINE#         818
  C:0534H         LINE#         819
  C:0536H         LINE#         820
  C:0538H         LINE#         821
  C:053AH         LINE#         823
  C:053DH         LINE#         824
  C:053FH         LINE#         825
  C:0540H         LINE#         829
  C:0542H         LINE#         830
  C:0543H         LINE#         831
  C:0545H         LINE#         832
  C:0546H         LINE#         835
  C:0548H         LINE#         836
  C:054AH         LINE#         837
  C:054CH         LINE#         838
  C:054DH         LINE#         841
  C:0550H         LINE#         842
  C:0552H         LINE#         843
  C:0553H         LINE#         844
  C:0555H         LINE#         845
  C:0557H         LINE#         846
  C:0559H         LINE#         847
  C:055BH         LINE#         848
  C:055DH         LINE#         849
  C:055FH         LINE#         850
  C:0561H         LINE#         851
BL51 BANKED LINKER/LOCATER V5.01                                                      03/27/2012  18:03:32  PAGE 15


  C:0564H         LINE#         852
  C:0565H         LINE#         855
  C:0568H         LINE#         856
  C:0569H         LINE#         857
  C:056BH         LINE#         858
  C:056EH         LINE#         859
  C:056FH         LINE#         860
  C:0570H         LINE#         861
  C:0572H         LINE#         862
  C:0573H         LINE#         863
  C:0574H         LINE#         864
  C:0577H         LINE#         865
  C:0579H         LINE#         866
  C:057AH         LINE#         869
  C:057DH         LINE#         870
  C:057FH         LINE#         871
  C:0581H         LINE#         872
  C:0583H         LINE#         873
  C:0585H         LINE#         874
  C:0586H         LINE#         877
  C:0589H         LINE#         878
  C:058BH         LINE#         879
  C:058DH         LINE#         880
  C:058FH         LINE#         881
  C:0591H         LINE#         882
  C:0592H         LINE#         885
  C:0594H         LINE#         886
  C:0596H         LINE#         887
  C:0599H         LINE#         888
  C:059BH         LINE#         889
  C:059DH         LINE#         890
  C:059FH         LINE#         891
  C:05A1H         LINE#         892
  C:05A2H         LINE#         893
  C:05A4H         LINE#         894
  C:05A5H         LINE#         895
  C:05A8H         LINE#         896
  C:05AAH         LINE#         897
  C:05ABH         LINE#         901
  C:05ADH         LINE#         902
  C:05AFH         LINE#         903
  C:05B1H         LINE#         904
  C:05B3H         LINE#         905
  C:05B6H         LINE#         906
  C:05B8H         LINE#         907
  C:05BAH         LINE#         908
  C:05BBH         LINE#         909
  C:05BEH         LINE#         910
  C:05C0H         LINE#         911
  C:05C3H         LINE#         912
  C:05C5H         LINE#         913
  C:05C7H         LINE#         914
  C:05C9H         LINE#         915
  C:05CAH         LINE#         916
  C:05CCH         LINE#         917
  C:05CDH         LINE#         918
  C:05D0H         LINE#         919
BL51 BANKED LINKER/LOCATER V5.01                                                      03/27/2012  18:03:32  PAGE 16


  C:05D2H         LINE#         920
  C:05D4H         LINE#         921
  C:05D5H         LINE#         924
  C:05D7H         LINE#         925
  C:05D9H         LINE#         926
  C:05DCH         LINE#         927
  C:05DEH         LINE#         928
  C:05E0H         LINE#         929
  C:05E1H         LINE#         930
  C:05E3H         LINE#         931
  C:05E6H         LINE#         932
  C:05E8H         LINE#         933
  C:05EBH         LINE#         934
  C:05EDH         LINE#         935
  C:05EFH         LINE#         936
  C:05F0H         LINE#         939
  C:05F2H         LINE#         940
  C:05F4H         LINE#         941
  C:05F6H         LINE#         942
  C:05F8H         LINE#         944
  C:05FAH         LINE#         945
  C:05FCH         LINE#         946
  C:05FDH         LINE#         950
  C:05FFH         LINE#         951
  C:0601H         LINE#         952
  C:0603H         LINE#         953
  C:0605H         LINE#         954
  C:0607H         LINE#         956
  C:0609H         LINE#         957
  C:060BH         LINE#         958
  C:060DH         LINE#         959
  C:060FH         LINE#         961
  C:0611H         LINE#         962
  C:0613H         LINE#         963
  C:0615H         LINE#         964
  C:0617H         LINE#         965
  C:0618H         LINE#         968
  C:061BH         LINE#         969
  C:061CH         LINE#         970
  C:061EH         LINE#         971
  C:0620H         LINE#         972
  C:0622H         LINE#         973
  C:0623H         LINE#         974
  C:0626H         LINE#         975
  C:0628H         LINE#         976
  C:062AH         LINE#         977
  C:062BH         LINE#         980
  C:062DH         LINE#         981
  C:062FH         LINE#         982
  C:0631H         LINE#         983
  -------         ENDMOD        UC51ALL

******************************************************************************
* RESTRICTED VERSION WITH 0800H BYTE CODE SIZE LIMIT; USED: 0637H BYTE (77%) *
******************************************************************************

Program Size: data=8.0 xdata=0 code=1773
BL51 BANKED LINKER/LOCATER V5.01                                                      03/27/2012  18:03:32  PAGE 17


LINK/LOCATE RUN COMPLETE.  0 WARNING(S),  0 ERROR(S)
